:020000040800F2
:100000002807002089010008EB1D00087113000873
:10001000E91D0008E30200086F1E00080000000050
:10002000000000000000000000000000EF1D0008BC
:10003000E502000800000000ED1D0008F11D0008A9
:10004000A3010008A3010008A3010008A301000800
:10005000A3010008A3010008A3010008A3010008F0
:10006000A3010008A3010008A3010008A3010008E0
:10007000A3010008A3010008A3010008A3010008D0
:10008000A3010008A3010008A3010008A3010008C0
:10009000A3010008A3010008A3010008A3010008B0
:1000A000A3010008A3010008A3010008A3010008A0
:1000B000A3010008A3010008A301000875130008AC
:1000C000A3010008A3010008A3010008A301000880
:1000D000A3010008A3010008A3010008A301000870
:1000E000A3010008A3010008A301000800F002F822
:1000F00000F03AF80AA090E8000C82448344AAF188
:100100000107DA4501D100F02FF8AFF2090EBAE885
:100110000F0013F0010F18BFFB1A43F0010318473B
:10012000101E0000301E0000103A24BF78C878C1AD
:10013000FAD8520724BF30C830C144BF04680C60ED
:10014000704700000023002400250026103A28BF35
:1001500078C1FBD8520728BF30C148BF0B60704739
:100160001FB51FBD10B510BD00F058F81146FFF7C0
:10017000F7FF01F08DFE00F076F803B4FFF7F2FF11
:1001800003BC00F07BF8000009488047094800479D
:10019000FEE7FEE7FEE7FEE7FEE7FEE7FEE7FEE737
:1001A000FEE7FEE704480549054A064B7047000094
:1001B0006D1E0008ED00000828010020280700201F
:1001C00028030020280300204FF0000200B513464A
:1001D00094469646203922BFA0E80C50A0E80C5067
:1001E000B1F12001BFF4F7AF090728BFA0E80C5018
:1001F00048BF0CC05DF804EB890028BF40F8042B11
:1002000008BF704748BF20F8022B11F0804F18BF7D
:1002100000F8012B7047704770477047754600F033
:1002200029F8AE4605006946534620F0070085468A
:1002300018B020B5FFF7B6FFBDE820404FF000062C
:100240004FF000074FF000084FF0000B21F00701BE
:10025000AC46ACE8C009ACE8C009ACE8C009ACE801
:10026000C0098D4670470446AFF300802046FFF773
:1002700084FF000000487047C40000200149182096
:10028000ABBEFEE7260002007047000070B50446D2
:1002900000688168C943C90717D1816821F001014D
:1002A000816000F0C9FA05460AE000BF00F0C4FA18
:1002B000401B022804D920688068C043C00706D0CC
:1002C00020688068C043C007F0D0002070BDA06ADD
:1002D00040F01000A062E06A40F00100E0620120FE
:1002E00070BDFEE770470000F8B50024009490F858
:1002F00024202546012A12D0012280F824204A68B1
:100300001F23072A0DD20668776B521E02EB82026A
:1003100093409F430B6893401F43776319E002208B
:10032000F8BD06680D2A0AD2376BD21F02EB820293
:1003300093409F430B6893401F43376309E0F76A7C
:100340000D3A02EB820293409F430B6893401F4398
:10035000F7620A68072306680A2A0AD3F7680A3A86
:1003600002EB420293409F438B6893401F43F76028
:1003700008E0376902EB420293409F438B68934049
:100380001F4337610A68102A01D0112A20D1124B6D
:1003900002689A4217D193681B0219D4936843F4F8
:1003A000000393600968102912D10C490C4A0968AE
:1003B000B1FBF2F101EB8101490000E0491E00911F
:1003C0000029FBD104E0816A41F02001816201240F
:1003D00080F824502046F8BD002401400C00002085
:1003E00040420F002DE9F0414FF0000704003D4668
:1003F0007ED0A06A002628B9E66284F824602046F0
:1004000000F07EF82046FFF741FFA16A01F01001DD
:10041000014304D0A06A40F01000A06268E0A16A25
:1004200021F4885141F00201A1626268E169237BF5
:100430000A4347EA43010A43A1684FF48077B9426F
:1004400008D0012906D0002194F814C0BCF1010F96
:1004500002D00AE03946F7E7F3B1A36A43F020037C
:10046000A362E36A43F00103E3622368D3F804C0A4
:100470002CF4694C4CEA010CC3F804C02368996859
:10048000DFF870C001EA0C0111439960A168B9421C
:100490000BD0012909D00CE0DFF85CC0A3690CEB9C
:1004A00043330B4343F40061DFE7218A0D05A5F5D3
:1004B00080152168CB6A23F470032B43CB6221683B
:1004C00089680E4B1940914208D1E662A16A21F079
:1004D000020141F00101A162BDE8F081A06A20F0B3
:1004E000020040F01000A062E06A40F00100E0620B
:1004F0000120F1E7FDF7E1FF00E0FFFFFE0E1FFF27
:1005000010B586B0002100910191029103911A4C1F
:1005100003681A4903221A48A34211D18B6943F494
:1005200000738B618B6903F4007304938B6943F050
:1005300004038B61896901F004010491012113E036
:10054000104CA34215D18B6943F480638B618B6996
:1005500003F4806304938B6943F004038B6189691E
:1005600001F0040104910221CDE90012694600F076
:100570006DF806B010BD00000024014000100240DC
:10058000000801400028014010B590F82110002417
:10059000022903D00421816301243DE001680A6837
:1005A00022F00E020A6001680A6822F001020A6065
:1005B0001A4A0168914201D1012121E0174A1432FF
:1005C000914201D110211BE0144A2832914201D1FD
:1005D000891515E0114A3C32914201D189140FE08E
:1005E0000E4A5032914202D14FF4803108E00B4A5A
:1005F0006432914202D14FF4801101E04FF08071DA
:10060000064A083A5160012180F82110002180F843
:100610002010416B01B18847204610BD0800024000
:1006200090F821007047000070B5044600F004F90E
:100630000546601C02D004480078044400F0FCF831
:10064000401BA042FAD370BD000000202DE9F84FF6
:10065000DFF8B8910024A9F1040B23460F2709F114
:10066000040AABF1040EC9E00125A5402A40AA42C4
:100670007DD1674ED1F804C0ACEB0608B44532D04A
:1006800014DCBCF1030F3AD009DCBCF1000F2AD016
:10069000BCF1010F1CD0BCF1020F31D11DE0BCF147
:1006A000110F17D0BCF1120F2AD119E0B8F5881F2D
:1006B00019D006DCB8F5803F15D0B8F5801F1FD1E2
:1006C00011E0B8F5001F0ED0B8F5041F18D10AE0EC
:1006D000CB6815E0CB681B1D12E0CB6808330FE038
:1006E000CB680C330CE08B682BB1012B4FF0080367
:1006F00003D0456104E0042302E0056100E000232B
:10070000FF2A01D8064601E000F104064FEA8405FD
:1007100001D9A5F12005D6F8008007FA05FC28EAE2
:100720000C0803FA05F548EA0508C6F800804D688C
:10073000ED0062D5374DAE6946F00106AE61AD6998
:1007400024F0030605F001050095334D06EB050C7A
:10075000DCF80850A607360F07FA06F825EA080560
:10076000DFF8B880404503D14FF0000817E044E0BF
:10077000DFF8AC80404502D14FF001080FE0DFF810
:10078000A480404502D14FF0020808E0DFF89880CD
:10079000404502D14FF0030801E04FF0040808FA89
:1007A00006F848EA0508CCF808804D68D9F80060DA
:1007B000ED024D4601D5164300E096432E604D688C
:1007C000DAF80060AD02554601D5164300E09643C5
:1007D0002E604D68DBF80060AD035D4601D5164321
:1007E00000E096432E604D68DEF80060ED0375462C
:1007F00001D5164300E096432E60641C0D682A461E
:10080000E5407FF431AFBDE8F88F000008040140F7
:1008100000001110001002400000014000080140DB
:10082000000C014000100140001401400AB10161B8
:1008300070470904FBE7000001488068704700002A
:1008400000000020704770472DE9F0470268002142
:100850005368C66A90F83E4090F83D50102C12D074
:10086000402C10D0046C002C7DD05469E443A607C2
:100870007AD4DE43B60577D4036C03B19169BDE841
:10088000F04701F051B9976951694FF42A0CC943F7
:100890005FEAC1784FF02A4904D066452AD04E4518
:1008A00028D010E0DE43B6050DD4C16A614501D100
:1008B000012103E0C16A494501D10821C162BDE8B7
:1008C000F04701F097B80E0716D4DE43B60513D4EF
:1008D000416CC9B21161416B09B1896A29B9816B57
:1008E000002907D0896A002904D00068416841F4D2
:1008F00000614160BDE8F0878E0706D4DE43B6058F
:1009000003D4BDE8F04700F0C9BFFE435268760744
:100910004FEA02521DD4002AECDB0A0608D4DA435F
:10092000520505D4490705D5BDE8F04700F05ABF88
:100930004907DFD4D9438905DCD4212D05D0402CCB
:10094000D8D1BDE8F04701F09BB8BDE8F04700F012
:1009500007BF002ACEDB4A060BD4DA43520508D47F
:10096000490708D501E00DE00EE0BDE8F04700F0D2
:1009700083BE4907BED4D9438905BBD4BDE8F0473F
:1009800000F010BE916970E7E10606D4D9438905ED
:1009900003D4BDE8F04701F0EBB82821212D27D082
:1009A000292D25D0650655D4DD436D0552D4640745
:1009B00052D590F83D30448D002C9BD01269446A8A
:1009C0002270426A521C4262428D521E4285428D02
:1009D000002A8FD12A2B8DD10268536823F48063BB
:1009E00053602222026380F83D1000F041F981E754
:1009F000250623D4DD436D0520D4640720D590F867
:100A00003D30448D002CF2D0446A24781461426A4F
:100A1000521C4262428D521E4285428D002AE6D10E
:100A2000292BE4D10268536823F4806353602122A8
:100A3000026380F83D1000F01CF95BE76107D6D433
:100A4000D9438905D3D4418D0029D0D0416A097892
:100A500011610AE06107CAD4D9438905C7D4418D21
:100A60000029C4D01169426A1170416A491C41626F
:100A7000418D491E41853DE77047000070B5040077
:100A800025D094F83D00002520B984F83C5020463C
:100A900000F0B8F8242084F83D002068016821F0B7
:100AA000010101602068016841F400410160206893
:100AB000016821F40041016000F080FA4A4A61684F
:100AC000914201D8494900E04949884201D20120B8
:100AD00070BD48492368B0FBF1F15E6826F03F061F
:100AE0000E435E606368934206D94FF49673594390
:100AF0004FF47A73B1FBF3F12368491C1E6A26F0A8
:100B00003F0631431962616891420AD84900401E8C
:100B1000B0FBF1F0401CC0F30B0004281ED20420EF
:100B20001CE0A368F3B301EBC10202EB0116421E05
:100B3000B2FBF6F2521C42F48042120549D093B344
:100B400001EBC10202EB0111401EB0FBF1F0401CB1
:100B5000C0F30B0040F4804040F400402168CA69B3
:100B60004CF6FF739A431043C861D4E90710014360
:100B70002068026822F0C00211430160D4E9030139
:100B800001432068826848F2FF339A431143816031
:100B9000D4E9050108432168CA6822F0FF02104326
:100BA000C86001E00EE016E02068016841F0010134
:100BB00001602564202084F83D00256384F83E50C0
:100BC000002070BD01EB4106421EB2FBF6F2521C42
:100BD000B3E70120C2E701EB4101401EB0FBF1F099
:100BE000401CC0F30B00B7E7A086010080841E0004
:100BF00000093D0040420F00704770477047704742
:100C00007047000010B586B000210091019102915B
:100C1000039100681349884222D1134CA06940F027
:100C20000800A061A069694600F008000490C02097
:100C3000009012200190032003900C48FFF706FD5E
:100C4000E06940F40010E061E069002200F4001067
:100C5000049011461F2000F073F81F2000F062F886
:100C600006B010BD0054004000100240000C0140CE
:100C7000704770470248816802781144816070476C
:100C800000000020074810B5016841F01001016024
:100C9000032000F075F80F2000F006F800F024F8AB
:100CA000002010BD0020024070B50D4D04464FF4E9
:100CB0007A712878B1FBF0F00A490968B1FBF0F0CD
:100CC00000F042FB48B9102C07D200222146501EEA
:100CD00000F036F800206C6070BD012070BD00008F
:100CE000000000200C0000200C4808B5816941F08C
:100CF00001018161816901F001010091C16941F047
:100D00008051C161C06900F0805000900448416882
:100D100021F0E06141F00071416008BD0010024027
:100D200000000140002809DB00F01F020121914072
:100D30004009800000F1E020C0F800117047000079
:100D4000F0B40E4B1B680C46C3F30223C3F1070536
:100D5000042D00D90425191D072901D2002300E024
:100D6000DB1E012606FA05F1491E214099409E40EE
:100D7000761E16403143F0BC01F07AB80CED00E06D
:100D8000064900F0070208684FF6FF03184040EAE2
:100D90000220034A10430860704700000CED00E099
:100DA0000000FA052DE9F84305460078354CC007E8
:100DB00054D0E0690026C00008D4E06940F08050BB
:100DC000E061E069012600F0805000902E48016843
:100DD000C90512D40168804641F480710160FFF7B3
:100DE0002BFD074605E000BFFFF726FDC01B64286A
:100DF00023D8D8F80000C005F6D5206A10F440705A
:100E000021D0A98801F4407181421CD0206A1F4979
:100E1000012220F440700A6000220A602062C007AC
:100E200011D0FFF709FD074641F2883808E000BFFE
:100E3000FFF702FDC11B414502D90320BDE8F8833D
:100E4000206A8007F4D5206A696820F4407008435E
:100E500020621EB1E06920F08050E06128788007B0
:100E600005D56068A96820F4404008436060287890
:100E7000C00605D56068E96820F48000084360601A
:100E80000020DBE7001002400070004040044242B6
:100E90002DE9F0470F46050061D0434E306800F061
:100EA0000700B84209D2306820F0070038433060AC
:100EB000306800F00700B84251D128683B4C8107E8
:100EC00012D5400703D5606840F4E0606060287880
:100ED000000703D5606840F4605060606068A968EE
:100EE00020F0F000084360602878C00728D06868C8
:100EF000012810D02168022810D0890700292EDA95
:100F0000616821F0030101436160FFF795FC8046B1
:100F100041F288390DE021688903EFE78901EDE7A7
:100F2000FFF78AFCA0EB0801494502D90320BDE880
:100F3000F0876068696800F00C00B0EB810FEFD1BA
:100F4000306800F00700B8420BD9306820F0070085
:100F500038433060306800F00700B84201D001200B
:100F6000E5E72878400705D56068E96820F4E06087
:100F7000084360602878000706D56068296920F476
:100F8000605040EAC100606000F028F86168084ADB
:100F9000C1F30311515CC840064908600648006867
:100FA000FFF782FE0020C2E700200240001002404E
:100FB000161F00080C00002004000020044805490A
:100FC00000684968044AC1F30221515CC840704777
:100FD0000C00002000100240261F00080E4A516835
:100FE0000E4801F00C03042B11D0082B0FD10C4834
:100FF000C1F38343C903C05C0AD55168084AC1F3F1
:101000004041921E515C054A5043B0FBF1F07047DD
:1010100004494843704700000010024000127A0063
:10102000061F000800093D002DE9F84F040070D0AC
:101030002078C04DC00749D06868C0F381000128FE
:1010400007D06868C0F38100022809D16868C0032E
:1010500006D52868800339D560680028E7D035E0D8
:101060006068B0F5803F0BD010B1B0F5A02F11D063
:10107000286820F480302860286820F4802002E06E
:10108000286840F480302860606890B1FFF7D4FB96
:1010900006460AE0286840F480202860F0E700BF98
:1010A000FFF7CAFB801B642873D828688003F7D534
:1010B0000CE0FFF7C1FB064605E000BFFFF7BCFBF5
:1010C000801B6428F0D828688003F7D420789A4ED3
:1010D00080074FF001094FF0000839D5686810F01B
:1010E0000C0F07D06868C0F38100022809D1686836
:1010F000C00306D42868800714D52069012808D1C8
:1011000010E02069B0B1C6F80090FFF795FB0746E4
:1011100005E00AE1FFF790FBC01B0228C4D828684D
:101120008007F7D52868616920F0F80040EAC1001F
:1011300028600DE0C6F80080FFF77EFB074604E05C
:10114000FFF77AFBC01B022823D828688007F7D452
:10115000207800072CD57948A169D9B1C0F8009052
:10116000FFF76AFB074604E0FFF766FBC01B022897
:101170000FD8686A8007F7D571484FF4FA510068B4
:10118000B0FBF1F0009000BF0098411E0091FAD230
:101190000EE080E0C0F80080FFF74EFB074604E059
:1011A000FFF74AFBC01B022875D8686A8007F7D48E
:1011B0002078400760D5E8690027C00008D4E869B6
:1011C00040F08050E861E869012700F0805000900D
:1011D0005C480168C90513D40168834641F48071F5
:1011E0000160FFF729FB824606E000BFFFF724FB02
:1011F000A0EB0A0064284ED8DBF80000C005F5D546
:10120000E06801280AD008B1052813D0286A20F028
:1012100001002862286A20F0040002E0286A40F0F9
:1012200001002862E06841F2883B98B1FFF704FBB7
:1012300082460BE0286A40F004002862EEE700BF17
:10124000FFF7FAFAA0EB0A0159455AD8286A800735
:10125000F6D50CE0FFF7F0FA824605E0FFF7ECFA6E
:10126000A0EB0A0159454CD8286A8007F6D41FB173
:10127000E86920F08050E861E06988B36968C1F3EB
:101280008101022944D00228C6F8608004D0FFF70B
:10129000D3FA044638E034E0FFF7CEFA074604E01C
:1012A000FFF7CAFAC01B02282BD828688001F7D4A0
:1012B000206AB0F5803F05D16868A16820F400304D
:1012C00008436860D4E908010843696821F474118F
:1012D00008436860C6F86090FFF7AEFA044606E07F
:1012E00025E000BFFFF7A8FA001B022809D82868EC
:1012F0008001F7D51BE000BFFFF79EFA001B022814
:1013000002D90320BDE8F88F28688001F4D40EE0EC
:101310000128F7D06868226A00F48031914204D134
:10132000616A00F47010884201D00120EAE70020D1
:10133000E8E7000000100240000042428004424200
:101340000C0000200070004010B5401EB0F1807FFE
:1013500001D3012010BD4FF0E02460610F21601720
:1013600000F086FD0020A06107202061002010BD54
:10137000FEE700000148FFF767BA00007000002098
:1013800038B5406A002190F83D202B4B46F2A81456
:101390001B68B3FBF4F3C3EBC30303EB83030093BA
:1013A0003BB15B1E009303681B689B0505D5009B42
:1013B000F6E7036C43F020030364436B03B19962C7
:1013C000836B03B1996203681C6824F480641C6019
:1013D0004185436B03B15963836B03B15963036860
:1013E0001C6824F001041C6090F83D402023602C10
:1013F0000BD0282434EA02020FD080F83D3080F868
:101400003E1000BFFFF738FB38BD80F83D3080F854
:101410003E100164FFF716FA38BD0268136843F006
:10142000010313600268136843F48063136001636F
:1014300080F83D40E6E700000C00002000684169AC
:10144000C943090601D400210161704770B5044603
:1014500090F83D0094F83E10102901D0402906D1A3
:10146000222804D121680A6822F400620A60282137
:1014700031EA00024FF000054FF0200626D0216827
:101480004968090505D4602803D084F83D6084F8D4
:101490003E50256320684168090537D5416821F42D
:1014A00000614160606B90F821203C49012A11D015
:1014B0004163606BFFF768F838B32068016821F07A
:1014C0000101016084F83D60606B1CE0256384F8D5
:1014D0003D10DFE7A06B4163A06BFFF755F8A0B1AB
:1014E00020684169C943490605D40069616A0870EA
:1014F000606A401C60622068016821F0010101609F
:1015000084F83D60A06B416B884710E094F83D1073
:10151000602910D04169C943490605D40069616A50
:101520000870606A401C60622046FFF7A5FA206CD4
:10153000C1071CD115E084F83D6025644169C943A9
:10154000490605D40069616A0870606A401C6062DF
:101550002068016821F0010101602046FFF772F95F
:10156000E5E7810703D4410701D4000704D52068CB
:10157000416821F4E061416094F83D00216C490725
:101580000BD5282809D10648E062256384F83D6020
:1015900084F83E502046FFF72FFB70BD81130008F2
:1015A0000000FFFF10B5C26A438D0168042B06D00E
:1015B000438D032B08D0438D022B1DD012E04A68C7
:1015C00022F480624A600CE04B6823F480634B6035
:1015D000042A06D0022A04D001680A6822F4806234
:1015E0000A6001680969426A1170416A491C4162D6
:1015F000418D491E418510BD012A30D0102A2ED0C0
:10160000042A30D0022A2ED00A6842F400720A60FE
:1016100001680969426A1170416A491C4162428D40
:10162000521E4285026812690A70416A491C416271
:10163000418D491E418501684A6822F440724A6022
:10164000202180F83D1090F83E200021402A80F8AB
:101650003E100CD012210163FFF7CFFA10BD0A68CB
:1016600022F48062D3E70A6842F48062CFE7016324
:10167000FFF7C5FA10BD000038B590F83D102229DB
:101680000FD1418D03290DD901680969426A117092
:10169000416A491C4162418D491E4185418D0329A2
:1016A00006D038BDC26A022A02D0012906D029B16B
:1016B0000068416821F48061416038BD274946F2E5
:1016C000A81300220968B1FBF3F101EB810100913D
:1016D00001682023009C641E009422D00C68A4059D
:1016E000F8D40C6824F480640C6001684C6824F41D
:1016F000E0644C6001680969446A2170416A491CD0
:101700004162418D491E418580F83D3090F83E1080
:1017100080F83E2040291DD012210163FFF76DFAA9
:1017200038BD046C44F0200404644C6824F4E06484
:101730004C6001680969446A2170416A491C416230
:10174000418D491E418580F83D3080F83E20FFF7ED
:1017500093F938BD0263FFF752FA38BD0C00002040
:1017600010B5C26A90F83D1021290BD1418D51B1BD
:10177000416A026809781161416A491C4162418DE0
:10178000491E418510BD20230021082A13D0202A9C
:1017900011D012F5803F0ED00268546824F4E06442
:1017A00054601122026380F83E1080F83D3000BF83
:1017B000FFF724FA10BD0268546824F4E064546012
:1017C0000268146844F400741460016380F83D30CA
:1017D00090F83E2080F83E10402AE9D1FFF710FA39
:1017E00010BD000010B590F83D1090F83E30C26A70
:1017F000048DB4B1212903D0402B11D122290FD15E
:10180000418DE1B390F83E10402942D0416A026810
:1018100009781161416A491C4162418D491E418527
:1018200010BD2129E8D120230021082A13D0202A25
:1018300011D012F5803F0ED00268546824F4E064A1
:1018400054601122026380F83E1080F83D3000BFE2
:10185000FFF7D4F910BD0268546824F4E0645460C2
:101860000268146844F400741460016380F83D3029
:1018700090F83E2080F83E10402AE9D100E002E0D6
:10188000FFF7BEF910BD0068416821F48061416036
:1018900010BDBDE8104000F0F3B8000078B590F836
:1018A0003E50C26A046B90F83D6000230168222E0E
:1018B00073D1066D0EB9402D6FD0056D1DB9056948
:1018C000B5F5404F1BD0458D95B3468D484D012E43
:1018D00020D0448D022C4DD00C6844F480640C6000
:1018E00001684C68240579D5AA4273D0012A71D0C9
:1018F000082A6FD0102A6DD0202A6BD06EE04A697A
:101900008A6900920A6842F480720A60016D491C7B
:10191000016578BDAA4214D10A6822F480620A6087
:1019200001684A68120504D50A6822F4806217E04B
:10193000FFE74A698A6900920A6842F400720A6005
:1019400050E0082A10D0202A0ED0122C0AD0042AE7
:1019500003D0022A01D0102AE6D10A6842F480623C
:101960000A603BE0012ADFD00A6822F480620A6044
:101970000168DEE7042A11D0022A0FD0102A0DD008
:101980000C6844F400640C6001684C698C69009434
:101990000C6824F480640C6008E025E00C6844F4D2
:1019A00080640C6001684C698969009101684C6829
:1019B000240517D5AA4207D0012A05D0082A03D04A
:1019C000102A01D0202A0DD14A6842F480524A6080
:1019D00008E0FFE74A6842F480524A6001684A69B9
:1019E00089690091036578BD48698869009078BD70
:1019F0000000FFFF90F83E10402910D00169B1F5BA
:101A0000804F19D0016DA9B3016D012910D1416C2E
:101A10005FF0F10201F4407142EAD11106E0016D7C
:101A20000029416C05D0C9B241F001010068016193
:101A3000704701F0FE01F9E790F83D102129416C53
:101A400009D0C9B241F0010102681161416B29B1AD
:101A5000896A49B902E001F0FE01F5E7816B0029CE
:101A6000E6D0896A0029E3D00068416841F400614A
:101A700041607047FFE7416CF02201F44071CBE711
:101A800010B590F83D10026D4AB1026D012A14D0D4
:101A9000026D022A16D0BDE81040FFF7CFBCC16C22
:101AA0000129816C02D0C1F3072108E00268C9B2A4
:101AB0001161016D891C016510BD816CC9B202689C
:101AC000116123E022291CD0428D0AB1212920D0A6
:101AD000428D002AF0D12129EED101684A6822F412
:101AE000E0624A6001680A6842F400720A600021FC
:101AF0000163202280F83D2080F83E10FFF780F837
:101B000010BD01680A6842F480720A60016D491CC8
:101B1000D1E7416A026809781161416A491C416252
:101B2000418D491E418510BD38B50C4690F83D20C9
:101B300000212825954302680B4605D0516991691B
:101B4000009180F83C3038BD556825F480655560BB
:101B5000E243540700D50121120601D5828900E035
:101B6000028B80F83C3092B2FEF76DFE38BD00006B
:101B7000F8B590F83D6004460068416821F4E061E2
:101B800041602068002541690091016841F0010130
:101B900001602068016821F480610160206841686B
:101BA000090520D5474F222E48D02A2E46D0616BFA
:101BB000096849686185618D19B1216C41F00401A2
:101BC0002164416821F400614160606BFEF728FDEB
:101BD000012808D0606B4763606BFEF7D5FC10B13D
:101BE000606B416B8847608D08B320684169C943C9
:101BF000490708D40069616A0870606A401C606225
:101C0000608D401E608520684169C943490608D43B
:101C10000069616A0870606A401C6062608D401EE5
:101C20006085608D18B1206C40F004002064206C49
:101C300000B32046BDE8F840FFF708BCA16B096877
:101C400049686185618D19B1216C41F004012164FD
:101C5000416821F400614160A06BFEF7E1FC0128BE
:101C6000C1D0A06B4763A06BFEF78EFC0028BAD0F2
:101C7000A06BB6E72A2E06D12563282084F83D0004
:101C80002046FEF7F5FF94F83D10202028290DD0BE
:101C9000216B222901D0222E07D1256384F83D0033
:101CA00084F83E502046FEF7E3FFF8BD0649E162A6
:101CB000256384F83D0084F83E502046FEF79CFFE3
:101CC000F8BD0000811300080000FFFF3EB50024AE
:101CD00011480094019402940E498460016001252A
:101CE0000573047505614FF460214460C161FEF71E
:101CF00079FB08B172B6FEE707200094CDE90150E8
:101D000069460548FEF7F0FA002801D072B6FEE7F2
:101D10003EBD000000240140100000203EB500241C
:101D200010480094019402940D498460016004738A
:101D30000475012505614FF460214460C161FEF71F
:101D400051FB08B172B6FEE70095CDE90154694632
:101D50000448FEF7C9FA002801D072B6FEE73EBD7E
:101D6000002801404000002070B586B000241C48C7
:101D70000094019402940394816941F010018161FF
:101D8000816901F010010491816941F020018161B4
:101D9000816901F020010491816941F004018161B0
:101DA000816901F004010491816941F008018161B8
:101DB00080690C4E00F008004FF40055049000229A
:101DC00029463046FEF732FD01200095CDE9010499
:101DD0000220039069463046FEF738FC06B070BD1D
:101DE0000010024000100140FEE7FEE77047704718
:101DF000FEF740BF30B593B028216846FEF7E4F9FE
:101E000014210AA8FEF7E0F9002501200F9510958E
:101E10001195010412958DE8230004904FF4E01011
:101E2000CDE90810022407946846FFF7FDF808B1D1
:101E300072B6FEE70AA90F2081E831004FF48060F6
:101E4000CDE90D0502210AA8FFF722F808B172B604
:101E5000FEE74FF4004011900F940FA8FEF7A2FF89
:101E6000002801D072B6FEE713B030BD7047FEE720
:101E70000907090E002804DB00F1E02080F80014B7
:101E8000704700F00F0000F1E02080F8141D70474B
:101E9000FEF7F8FEFFF7AEFFFFF766FF164815499D
:101EA0004FF4804201601549416000218160C0E922
:101EB000031241618161C1610162FEF7DFFD08B17A
:101EC00072B6FEE7FFF702FFFFF728FF0C4C4FF456
:101ED0000055012229462046FEF7A8FCC820FEF73F
:101EE000A3FB002229462046FEF7A0FCC820FEF7EF
:101EF0009BFBEEE70054004070000020A08601002C
:101F000000100140010202030405060708090A0B3C
:101F10000C0D0E0F10100000000000000000010268
:101F20000304060708090000000001020304000082
:101F3000501F0008000000201000000028010008C9
:101F4000601F00081000002018070000440100086E
:101F50000100000010000000000000000024F40058
:04000005080000ED02
:00000001FF
